:0C000E0020566572732E20312E30200029
:03000B000202727C
:10027200C0E0C0F0C083C082C0D075D010C2AF054C
:100282003AE53A70020539E53AB4E814E539B403BF
:100292000FE54E0475F03C8485F04EE4F539F53AED
:1002A200758A66758CFCD2AFD0D0D082D083D0F064
:0302B200D0E03267
:0300230002002EAA
:10002E00C0E0C0F0C083C082C0D075D018C2AC3062
:10003E009958C299C200AB24AA25A9269000011294
:10004E0003F1FFAB24AA25A9261203D66F70030273
:10005E0000F5AB24AA25A9261203D62402FFE43408
:10006E0000AB24AA25A9268F82F5831203F1FFF592
:10007E0099AB24AA25A9267401120420540FFFABB4
:10008E0024AA25A926120479805DC298AB21AA2242
:10009E00A9239000011203F104540FFFAB21AA22F1
:1000AE00A9231203D66F603FAB21AA22A923900089
:1000BE00011203F12402FF74003400AB21AA22A91D
:1000CE00238F82F583E59912048DAB21AA22A923F1
:1000DE009000017401120444540FFFAB21AA22A90F
:1000EE002390000112048DD2ACD0D0D082D083D018
:0400FE00F0D0E0322C
:03002B0002025975
:10025900C0D075C7AA75C7555387FBD2B575C7AA4C
:0902690075C755438702D0D0325D
:1001510043870875C7AA75C7555387FBC2B5E4F530
:1001610039F53A7521047522007523277524047524
:10017100250075263BAB21AA22A923900001120478
:100181008DAB21AA22A923E4120479AB24AA25A9C3
:1001910026900001E412048DAB24AA25A926E412BD
:1001A1000479C2007598D2758920758DE8D28ED2F6
:1001B100AC438901758A66758CFCD2A9D2BCD2AFD9
:1001C100D28C75C7AA75C755D2BFB2B579057A1851
:1001D1007B0290180612050F1201F6400A75C7AA94
:1001E10075C755D2BF80E5901805E0901809F01247
:0501F10002B580CE22E2
:1002B500C2ACC201AB24AA25A9269000011203F104
:1002C500FFAB24AA25A9261203D6FEB50704A20072
:1002D5005063AB24AA25A9269000011203F104540A
:1002E5000FFFAB24AA25A9261203D66F60529018DA
:1002F50009E0FFAB24AA25A9269000011203F1FE0F
:100305002402FD74003400AB24AA25A9268D82F5AC
:1003150083EF12048DAB24AA25A9269000011203B0
:10032500F104540FFFAB24AA25A92690000112045D
:100335008DD201800B901809E0FFF599D200D2010A
:05034500D2ACA2012270
:1001F600C201AB21AA22A9239000011203F1FFAB91
:1002060021AA22A9231203D66F6045C2ACAB21AA4C
:1002160022A9231203D62402FF74003400AB21AABC
:1002260022A9238F82F5831203F1FF901806120587
:1002360006EF120479AB21AA22A923740112042025
:10024600540FFFAB21AA22A923120479D2ACD20102
:03025600A20122E0
:10010200901800E0FEA3E0253AFFE5393EFE7C03AD
:100112007DE81204B18C4F8D50C3E550953AE54FFE
:1001220095395015C3E550953AE54F9539501F75ED
:10013200C7AA75C755D2BF80EBD3E550953AE54FB4
:0F0142009539400A75C7AA75C755D2BF80EB2201
:0600030043180205000E87
:0300000002034AAE
:0C034A00787FE4F6D8FD75815002039125
:1003D600BB020689828A83E0224003BB0402E7222D
:0B03E600400789828A83E49322E3220F
:1003F100BB020CE58229F582E5833AF583E02240D0
:1004010003BB0406E92582F8E622400DE58229F5C1
:0F04110082E5833AF583E49322E92582F8E2221B
:10042000BB020989828A83F8E028F0224003BB04DA
:100430000327F72240098A838982F8E4932822F867
:04044000E328F32298
:10044400BB020FF8E58229F582E5833AF583E028BB
:10045400F0224003BB0409C58229F8E58226F6226E
:10046400400AF8EA2583F583E9932822C58229F80E
:05047400E22582F222E6
:10047900BB020689828A83F0224003BB0402F72269
:040489005001F32209
:10048D00F8BB020DE58229F582E5833AF583E8F0A4
:10049D00224003BB0406E92582C8F6225005E92552
:0404AD0082C8F222ED
:1004B100BC000BBE0029EF8DF084FFADF022E4CC2F
:1004C100F875F008EF2FFFEE33FEEC33FCEE9DECF8
:1004D100984005FCEE9DFE0FD5F0E9E4CEFD22ED3E
:1004E100F8F5F0EE8420D21CFEADF075F008EF2F88
:1004F100FFED33FD4007985006D5F0F222C398FD79
:050501000FD5F0EA2215
:09050600E0FBA3E0FAA3E0F922F6
:09050F00EBF0A3EAF0A3E9F022ED
:10035600020151E493A3F8E493A34003F68001F26B
:1003660008DFF48029E493A3F85407240CC8C333A8
:10037600C4540F4420C8834004F456800146F6DF77
:10038600E4800B0102040810204080900003E47E04
:10039600019360BCA3FF543F30E509541FFEE4936C
:1003A600A360010ECF54C025E060A840B8E493A333
:1003B600FAE493A3F8E493A3C8C582C8CAC583CA5E
:1003C600F0A3C8C582C8CAC583CADFE9DEE780BE16
:0100090000F6
:00000001FF
